:100000005AC074C0EEC172C071C070C06FC06EC003
:100010006DC06CC06BC06AC069C068C067C066C094
:1000200065C005010900A1010508194B294B150000
:1000300027FFFF0000751095018102C00403090429
:100040001C034200690064006F00750069006C00C9
:100050006C0065002E006F007200670026034B00E5
:1000600076006100720074007300200044005200AA
:10007000530042002D003000310020005500530095
:1000800042001201100100000008C016EC0300013C
:10009000010200010902220001010080320904006E
:1000A000000103000000092101010001221A0007DC
:1000B00005810308000A11241FBECFE5D1E0DEBF91
:1000C000CDBF10E0A0E6B0E0EAE5F6E002C00590A2
:1000D0000D92A236B107D9F710E0A2E6B0E001C058
:1000E0001D92AB39B107E1F704D0B5C289CF80E0EA
:1000F000089580E395E70197F1F7479A1FBC8EB505
:1001000086608EBD21D0D09A80E197E22CE231E06A
:10011000F9013197F1F70197D9F7D0987894D39AEC
:10012000D298D79ADB98DF981AD08091700084FF1C
:10013000FBCF8CB59DB5909364008093630083E6FC
:1001400090E062E014D1F0CF919A8BB780618BBFC1
:100150008BE4809371008AE58093700008951F936B
:10016000CF93DF9390918100935097FDA5C020918C
:100170007E0080917D008D3209F09CC0983009F09E
:1001800099C0CCE0D0E0C21BD109CB57DF4F83EC44
:10019000809365008AE580936000109262008881F8
:1001A000807621F0CE01A3DF282F7BC09A811092A8
:1001B0006E008981882321F410926F0022E06BC0C9
:1001C000853019F49093820065C0863009F04EC0E6
:1001D0008B81813041F482E890E09093800080939D
:1001E0007F0022E13FC0823041F484E990E09093A7
:1001F000800080937F0022E235C08330F1F49923A0
:1002000041F48CE390E09093800080937F0024E0A1
:1002100029C0913041F480E490E090938000809375
:100220007F002CE11FC09230E1F48CE590E09093C8
:10023000800080937F0026E215C0813241F486EA77
:1002400090E09093800080937F0029E00BC0823281
:1002500041F482E290E09093800080937F002AE155
:1002600001C020E080E4809362001BC0883021F44C
:1002700021E084E890E011C0893019F49093840063
:1002800009C08A3011F421E006C08B3019F48BE4E8
:100290008093710020E08EE690E090938000809340
:1002A0007F008F81882321F48E81821708F4282F04
:1002B00020936100109281008091600084FF49C00A
:1002C000809161008F3F09F444C0182F893008F0F5
:1002D00018E0811B809361008091650098E8892770
:1002E00080936500112341F120917F0030918000BF
:1002F0008091620086FF0DC0A6E6B0E080E090E04D
:10030000F901E80FF91FE491ED9301961817C1F771
:1003100008C0912FD901E6E6F0E08D9181939150CC
:10032000E1F71150812F90E01F5F0196820F931F1C
:100330009093800080937F0086E690E0612F4DD0FF
:10034000612F6C5F6C3019F08FEF809361006093C8
:10035000600094E189B3837031F49150D9F7109221
:10036000820010927C00DF91CF911F9108951F931E
:10037000DC01162F8091700084FF07C0809171000E
:1003800098E889278093710003C08AE58093700004
:10039000912FE2E7F0E08D9181939150E1F782E7B0
:1003A00090E0612F1AD01C5F109370001F91089588
:1003B000A82FB92F80E090E041E050EA609530E04E
:1003C00009C02D9182279795879510F0842795274E
:1003D000305EC8F36F5FA8F30895EADF8D939D93B5
:1003E0000895CF93CFB7CF93C395C89BE9F7C89B28
:1003F00009C0C89B07C0C89B05C0C89B03C0C89B59
:1004000001C0A3C0DF93C0917E00DD27CB57DF4F33
:10041000C89B02C0DF91EBCF2F930F931F9309B3BB
:100420002FEF00FB20F94F933F9319B34FEF0127B4
:1004300000FB21F93BE031C04E7F012F19B3216051
:1004400028C0102F4D7F2260000009B329C04B7FC8
:100450002460012F000019B32BC019B3477F286017
:100460002AC04F7E09B320612CC04F7D19B3206292
:100470002FC04F7B09B3206432C0422709B3499390
:100480004FEF0000102710FB20F919B31370C9F1CA
:10049000297F91F2012700FB21F909B3237F89F21B
:1004A000315058F1102710FB22F919B3277E79F249
:1004B000012700FB23F92F7C81F209B3102710FBE1
:1004C00024F92F7971F200C019B3012700FB25F937
:1004D0002F7359F200C009B3102710FB26F9223000
:1004E00040F200C019B3012700FB27F9243028F699
:1004F0004F77206819B30000F9CF10E11ABF002729
:1005000019C03B503195C31BD04010E11ABF088180
:10051000033CF9F00B34E9F020917C001981110FB4
:100520001213EDCF4A81441F093641F10D3211F00B
:10053000013E29F7009383003F914F911F910F9146
:100540002F91DF91CAB7C4FD4FCFCF91CFBFCF91CD
:10055000189520918300222379F3109181001123B3
:1005600069F534306AF13093810020937D00109159
:100570007E003BE0311B30937E0022C00091810061
:100580000130E4F40AE54F7049F43091600034FD25
:1005900019C000936000C5E6D0E018C0309170002B
:1005A00034FD10C000937000C1E7D0E00FC0279564
:1005B000A8F45150A9F4220F0000F9CF4AE503C076
:1005C00042ED01C0432FC4E1D0E032E01AB3136022
:1005D000D89A1ABB0BB320E413E05F93012756E0CF
:1005E0000BBB279520F4515021F4220FF9CF01279E
:1005F00056E000003B5A0BBBD0F2279528F451502F
:1006000029F4220F0000F9CF012756E027950BBBF4
:1006100020F4515021F4220FF9CF012756E02991FF
:1006200033230BBB21F60C7F10918200110FC651B2
:10063000D0400BBB11F010937C0010E11ABF016099
:100640001AB31C7F402F4C7F5F9100C000C00BBBD2
:0A0650001ABB4BBB71CFF894FFCF2B
:02065A005AFF45
:00000001FF
